:100000004AC1189505C164C01895189503B601E05A
:1000100003BF03FC1895939402E008BF06E009BFF4
:10002000019691FE0FC00B2E8A0E011C06BE04E045
:1000300003B909E003BF03E20FBD02E08038900777
:1000400048F322C101E003B916BE8C01169507954D
:100050000230110560F071F444B005B086D038016B
:1000600045D030015527442776956795189502E4C9
:1000700007B91895E4B0F5B0E218F308E414F504F4
:100080001CF40A30110508F0C2989C01261B370B9E
:1000900083012CD00E181F08900104E610E026D032
:1000A00070012C193D09C20ED31E0AE010E01ED0CB
:1000B000E00CF11C112400E8E00EF11C2AF0EB1614
:1000C000F10420F0E9BC189519BC1895B9BD189534
:1000D000939404E009BF91FC06C008BF03EE0FBD76
:1000E00000EF06BF189500E406BF18951124002400
:1000F00000FD020E00FD131E1594079401FD020E73
:1001000001FD131E1594079402FD020E02FD131E3D
:100110001594079403FD020E03FD131E1594079416
:1001200004FD020E04FD131E1594079405FD020E36
:1001300005FD131E1594079406FD020E06FD131E01
:100140001594079407FD020E07FD131E15940794DE
:1001500010FD020E10FD131E1594079411FD020EE2
:1001600011FD131E15940794089500271127000C04
:10017000111C0616170618F4061A170A1260000C4E
:10018000111C0616170618F4061A170A1160000C3F
:10019000111C0616170618F4061A170A0068000C38
:1001A000111C0616170618F4061A170A0064000C2C
:1001B000111C0616170618F4061A170A0062000C1E
:1001C000111C0616170618F4061A170A0061000C0F
:1001D000111C0616170618F4061A170A0860000CF8
:1001E000111C0616170618F4061A170A0460000CEC
:1001F000111C0616170618F4061A170A0260000CDE
:10020000111C0616170618F4061A170A016008953D
:1002100008B602B7192D002009F001FC1395B39917
:100220002AC00A191B09A00EB11E0058134041F440
:10023000083730F0083820F48501037001FD0C6F99
:100240000058104015950695A00FB11F11B70CEF7F
:10025000A030B00728F00FEFA130B00730F41895A8
:10026000BE5F13950AF011BF1895B2501A9510375A
:1002700008F411BF18950A191B0961F0992351F070
:1002800001E0843F900708F0BC01C29A16BE90E0DE
:1002900080E017B81895112460E872E00FE701BFFD
:1002A00000E205BF09E008BB06E207BB08E005BBAA
:1002B00001E003BF00EE06BF08E009BF00E808B98F
:1002C00002E407B906EE06B907E304BBA0E0BFEFFE
:1002D00008EE13E0780180E090E078948895F89437
:1002E000081B190BC1F724B035B00FEF09BD03EEA1
:0A02F0000FBDC19A78948895FECFE7
:02000004008278
:02000000FAFE06
:02000004008476
:030000001E900748
:00000001FF
